:10000000860185018316AD28F82E8207D02BD32BCD
:10001000D62BD92BDE2BE32BEA2BF12B8207523484
:100020005834003444344434533420345234453446
:10003000463420344D3455344C3454340034203458
:1000400052344534463443344C344B3400344D340C
:1000500041345834203400344D3449344E34203443
:1000600000345334413456344534203454344F34FE
:1000700020344D3400345634613420340034563446
:1000800062342034003452344934543420344F34F0
:1000900046344634533445345434203400345334D5
:1000A000533442342034003441344D34203400344D
:1000B00043345734203400344C3453344234003405
:1000C0005534533442340034203453345934533487
:1000D000543445344D34203443344C344B340034A0
:1000E0002034443444345334203446345234453478
:1000F00051342034003453344134563449344E346E
:10010000473400344D3448347A34003423342034B6
:10011000203400343C343E342034003443344E34F4
:100120005334203434342E343034003442342034C8
:100130003D343E34203441340034413420343D34A5
:100140003E3420344234003455344E344C344F3431
:1001500043344B34453444340034063086002F3069
:100160008500813081008E309F009901F030980029
:1001700083128030980086168612061406100A3004
:100180009F00203084005030B026BA26DE24A030F4
:100190008B006C267F303A263130D51B36305726FF
:1001A000A130F600AD26761C4714B8254C26F60B78
:1001B000D2284A26A201AC1BF0293A18DD28DE24F9
:1001C000F524D0213B153C1BE928B21FFD283C1724
:1001D000EC28B21FFD283C135326033045269530EA
:1001E0003C1B97303A2607303C1F05304526CD3062
:1001F00054264025B21BFA28BB143C08C100063027
:100200002B02BC16031CBC123C08C106C11A3B15CC
:10021000BE1D11295D23B924BA1C1929BE113B1535
:1002200019293E1B1629BD1549249023B924BA1853
:10023000BE213E1F3B29B324BA183229B41B3329EF
:10024000BE1D202BBE0D5608FF00FE01FD01FC0166
:10025000CC250310BE0C4D08C4004E08C500412338
:10026000D0215329F524EE243E13D0213B156F25D0
:10027000B41B3829E328AE1F4E29C4303E1AC930BA
:10028000D72453260230452687303E1A8E303A2630
:1002900008304526AE1B4A29BB14A501B41B1B2BF5
:1002A000B324BA18BA29B724BA1C5B29BE0A3E1176
:1002B000D0213B15A5013B1A6129B01F76293B16B9
:1002C0006529B01F6D293B123B15C03054262030E4
:1002D0003B1A7E305726B01B6B29BC1E7329BB1DF1
:1002E000C121BB157929BB19C121BB11B524BA188D
:1002F000C1213B1D89293026BC1A8129BE19E8225B
:1003000085293E080339013A031DFA22B2253B1123
:10031000BB14391E9729AD3084003E087839550446
:100320008000840A560880003E1FCE24C026BB1CD5
:10033000E328721FE3286F25BE0D2A250310BE0C8B
:10034000AA21BB10F201E328E709E809E80F080039
:10035000E70A0800831618108312FE307C05031D7F
:10036000B7297D08C1007C0C410C99000800FF30C2
:10037000990008003E17CE243B15E328BE153B1517
:1003800008003E1FC829F524EE243E133B15D02952
:10039000CE243E1ACD293E16CE293E123B15F52419
:1003A0003B103E0803390319DB29BE1CDF293E1C24
:1003B0003B14BF30E029E701E8010516EA29C13006
:1003C00084000008E700840A0008E8003B18A42124
:1003D0003B1005128316181483123E08990008007A
:1003E000BE019F264A2603303A26A526A326DE0A0A
:1003F000A726D51B6C14B911B919E52A8E23C03074
:1004000054267830572631306F1836305726103042
:100410003A26B124BA1CFC29D5136F18D5175508F4
:100420008316AD0083124A26F12303309E245F30E9
:10043000D724F12313309E245B30D724AF30DB2444
:10044000FC238330542655303A263B15492490230B
:10045000A930D7243B192A25FC235730D724F12370
:100460004F3084007C3003253B19B225A930DB24B2
:10047000B124BA1C262AFC23AF30D7244A26F12304
:1004800005309E245B30D72489265F30D724BB30CB
:10049000DB244A2637303A2666303A26B919E52A4F
:1004A0004A2490232A25B124BA1C4E2ABB30D724D3
:1004B000A526A93084004F30032509309E24A126AB
:1004C0001430DA0004245B30D724B330DB244A260E
:1004D00018303A2661303A26B911B919E52A49246B
:1004E00090232A25B124BA1C6D2AB330D7244A267A
:1004F000B33084005B300325BB3084005F300325BC
:100500008126B730DB2453261D303A2600303A26A8
:1005100061303A26B911B919E52A4A2490232A25CF
:10052000B124BA1C8B2AB730D7244A2604300520C0
:1005300003309E245B30D72489265F30D724BF3018
:1005400084000008EE00840A0008EF00ED01EC01D1
:100550004A2640303A2637303A26B919E52A4A2445
:1005600090239F262A25B124BA1CAD2ABF308400CF
:100570006E088000840A6F088000C1308400000883
:10058000EE00840A0008EF00ED01EC01532649302B
:100590003A26B919E52A4A2490232A25B124BA1CFF
:1005A000C92AC13084006E088000840A6F08800068
:1005B0003913B6263916391FE52ABE114A26853069
:1005C00054266C303A26A31BE32ABA264A26DF2893
:1005D000F001D31BF0035408FF0753080318530F0F
:1005E000FE0770080318700FFD0770080318700FDE
:1005F000FC070800F001E71BF0036808FF07670825
:100600000318670FFE0770080318700FFD077008C6
:100610000318700FFC0708006608FF076508031839
:10062000650FFE0764080318640FFD0763080318CD
:10063000630FFC070800CE244A2622303A26BA155A
:10064000A526E20AA3261330DE00B911B919372B0B
:10065000A7265608EF008E233026CC256F08D6003B
:100660003E1B2B29482541232A25B324BA18E52A05
:10067000B41FBA11BA1DB41F262BF5244023DE2A5D
:10068000B916A9263E0803398316A0008312A130AB
:10069000D7245603D20005309E24A03084000530B4
:1006A000F50020306F07CE267830BE05A0308400DC
:1006B0000008BE04A130DB2408002208031908004A
:1006C0003C1B08003B15F600A201F61F7B2BF6131E
:1006D0007608D402031CD303D31F08005408B83E85
:1006E00053080318530F0B3E031808004830D4007A
:1006F000F430D30008007608D4070318D30AD31BBC
:1007000008005408483E53080318530FF43E031CD6
:100710000800B830D4000B30D30008003C16912BF1
:100720002E243C1B080022080319A52BF600A20169
:100730006B083C1A03010520F61B8726F613942547
:100740003C1AA42BF60B9F2B3B153C12CB236F08B6
:100750005E026E08031C6E0F5D026D08031C6D0FB8
:100760005C026C08031C6C0F5B020318B92B5B3036
:10077000DB246F0862026E08031C6E0F61026D08B5
:10078000031C6D0F60026C08031C6C0F5F02031CDE
:10079000CB2B5F30DB248030EC06DF06DB06080065
:1007A0000130D200F82B0A30D200F82B6430D2008E
:1007B000F82BE830D2000330D100F92B1030D200F2
:1007C0002730D100F92BA030D2008630D100013083
:1007D000D000FA2B4030D2004230D1000F30D00090
:1007E000FA2B8030D2009630D1009830D000FA2B0E
:1007F000D101D001CF0108006C30840057300325AF
:10080000A726AD264714052CAD262030F70003108F
:10081000EF0DEE0DED0DEC0DCA0DC90DC80DC70D98
:100820000318152CD71FEF0A172CD71BEF0A6F1CC4
:10083000A3256F182A24F70B072C0310EF0DEE0DDC
:10084000ED0DEC0DC71B272CD71FEF0A0800D71B97
:10085000EF0A08008526A32585260800A61D0800A6
:100860000E3054266B308400063000020318013E1F
:10087000C53C542622080319452CA21B800A801966
:100880008003A21F8003801B800AA201A619322CBC
:100890007A2E3D153C1B0800A624BA1C9C2CB911CD
:1008A0003D14A130D724A7260330F100381F682C4F
:1008B0003D195C2CBD14F10330263125B91D632C84
:1008C000A130DB249C2CA624BA1C5E2C381B902C57
:1008D000B81E702C3D1A5E2C3D160630F1005C2CC3
:1008E000710803195E2C71033D1A7D2C6C30840055
:1008F0004F3003250A309E2406300520A530D7242A
:1009000038089E24A53084004F30032594253D1AD5
:100910008E2C6C086D046E046F04031DF1035C2CB7
:10092000BD188926BD1D9C2C832630260C237C30C7
:10093000DB24832639163B15BD010800013EF40077
:10094000A726A32C9425F40BA22C08003A19AD2C51
:100950000630360203183A15CA2C360803193A1124
:10096000CC2C2D30BA2C3530BA2C3130BA2C333057
:10097000BA2C2F3084000008C10084030002000854
:10098000840A80000318CC2C4108063C0318CC2CA8
:100990004108463CBA14031CBA100800C3303E1E7E
:1009A000C83084003E0E30396B048000040AC10058
:1009B0006C308400042D84006C30032D0330BE05A0
:1009C000AD30840000088039D50000087839BE04B5
:1009D000840A5630C1001530F700062DB33084006C
:1009E0005B30C1000830F700062DC3303E1EC83012
:1009F000840000080F39EB007830BE05000E033983
:100A0000BE04840A6C30C1000430F7000008C30043
:100A1000040AC2004108840043088000040AC1009F
:100A200042088400F70B062D0800AD262030F700A1
:100A30007F0CFC0CFD0CFE0CFF0C0318A325C70C4F
:100A4000C80CC90CCA0CCB0CCC0CCD0CCE0CF70BC3
:100A5000182D080030260C23BC10FC1F312DBC14AF
:100A60008B26CD252B26C23054260008572607306A
:100A700075022E3003195726840AF50B352D56269C
:100A800073303D1877303C1B7B303A26BC10080091
:100A9000893054264D0857264E0857260800BC10AA
:100AA000D31F542DBC146925CD254A308400053050
:100AB000F5008A30542600085726043075022E307F
:100AC00003195726840AF50B5B2DBC186925BC1049
:100AD0000800D309D409D40F0800D30A080053260C
:100AE0005230BC1A54305726013045262A303E1B5E
:100AF0007C2D2C303E1E30303A263E1F832D44087C
:100B0000572645085726013045263E083E073E0732
:100B10003E070F39453E3A2601304526063EBE19AE
:100B20004F25BE1D452608005208EF07510803183F
:100B3000510FEE0750080318500FED074F08031828
:100B40004F0FEC0708005A08CA0759080318590F35
:100B5000C90758080318580FC80757080318570F34
:100B6000C7070800FC1B8B261525C701D51B47149A
:100B70002830F5008B13C70CC80CC90CCA0CCB0C61
:100B8000031C86130318861786168612F50BBB2DD9
:100B9000061406108B1708003C15AD262030BE1930
:100BA0001030F600BE19E22DE62D2B26033000078B
:100BB000C100C11DDD2D783E8000840AF50BD62DC5
:100BC000BE1DE62D530DD40DD30DEB2D7C0DFF0D69
:100BD000FE0DFD0DFC0DCE0DCD0DCC0DCB0DCA0DBA
:100BE000C90DC80DC70DC60DF60BD52D3C102B2613
:100BF0003D1EFE2D750871020318092E0008031909
:100C0000052E303E80003C140B2E3C18012E0408AB
:100C1000F60020308000840A08303C190130BE19EB
:100C20000530750203193C14F50BF82D3C11BD1865
:100C3000262EBC18262EBE1D080054085304031986
:100C40000800760884002B308000080076088400B5
:100C50002D3080000800463084000930F50008007F
:100C60006C08FC006D08FD006E08FE006F08FF00B8
:100C700008000A14C1000E20FF390319422E57261E
:100C8000410A3A2E0A1008001030F4005626F40BE0
:100C9000462E0800013054260830F400030168266F
:100CA000F40B4E2E080080300513582E2030051707
:100CB000C3008B135F26C30E5F268B1708000F300F
:100CC00086054308F0398604CE308615000086116B
:100CD000013E031D682E08007C267C267C262830D9
:100CE00086000513642628305426083054264A26E8
:100CF000063054260C30542E3830860005136426F6
:100D00004C2E5F308C2E63308C2E57308C2E4F3013
:100D10008C2E6C308C2E7C3084008009840A8009F3
:100D2000840A8009840A8009800F08008403800FE8
:100D300008008403800F08008403800A08006330E1
:100D4000AA2E5730AA2E5B30AA2E5F30AA2E6C3006
:100D5000AA2E4F3084000430B02E46308400093073
:100D6000F5008001840AF50BB12E0800B916163083
:100D7000BB2EB9162030F500AD3084000030CE2EE9
:100D8000B9160230F500AD3084000030CE26B91619
:100D90000A30F500C33084001630CE2E83169B0037
:100DA0008312B91ADD26F326800083169B0A83126C
:100DB000840AF50BD12EB9120800F326000203199C
:100DC000F12E00088C1383169A001C158B135530D6
:100DD0009D00AA309D009C148B1783128C1FEE2E51
:100DE00039173912080083161C141A0883120800D8
:100DF000FA00030EF90083120608FB00E0308600BB
:100E000085179F110310F80C0310F80C1F08C03948
:100E1000F8049F155530780503193910553A031910
:100E20003914AA3078050319B910AA3A0319B9146C
:100E30003919262F391C262F2108A200B91CA21708
:100E40002630A100A5010530A400A30139113918ED
:100E50003915210BA100721FF20AA00BA32FA015B8
:100E60001F0E061686120C39A7001F0E9F110C3993
:100E7000A8001F0886160613C039A8041F089F156E
:100E8000C039A9001F0E061786130C39A9041F0EBE
:100E90009F110C39AA001F0886178513C039AA04B0
:100EA0001F089F15C039A6001F0E0C39A6043A1062
:100EB000360FB600030129198030281B8130291B09
:100EC00082302A1B8330A81B8430A91B8530AA1BC3
:100ED0008630A8198730A9198830AA1989302819AD
:100EE000A0302A19C030003E031DB8000319B60116
:100EF000260427040319802F0530A400A3013A1407
:100F0000B813300FB000271DB001320FB200A61F7A
:100F1000B201340FB400A71DB4012E0FAE00261F7E
:100F2000AE012C0FAC00261DAC012B0FAB00851AB7
:100F3000AB01250FA500FE3C03193916A3030319C5
:100F4000A4030319B9157B088600790E8300FA0EF5
:060F50007A0E0B110900EE
:02400E00503F21
:10420000900001001700DC006500DE000300DF0005
:10421000D20040000000000000000000000000008C
:10422000000000000500DC0003002000000000008A
:10423000A0003700A000000000006B0093001000F9
:104240000000000098009600800001000000990026
:104250005900D000020000009A001D002000030059
:1042600000009A00E0007000030000009B00A30023
:10427000C000020000009C00670010000100000068
:104280009D002A006000000000009D00ED00B000CD
:10429000030000009E00B1000000020000009F002B
:1042A0007400500003000000A0003700A0000000D0
:1042B0000000A000FA00F00000000000A100BE0015
:1042C000400000000000A2008100900000000000FB
:1042D000A3004400E00000000000A400080030003B
:1042E00000000000A400CB00800000000000A5003A
:0E42F0008E00D00000000000A600520020004A
:00000001FF
